:030000000219FDE5
:03000B000200AA46
:03002B0002019936
:03005B0002034F4E
:0300730002033550
:1000800002030406080C10182030406080040608A3
:100090000C10182030406080A0C000070F1F3F0DDB
:1000A0000D0403060D0503030202C2AF306308C24C
:1000B00063857C8AD2AF32C0D0C0E0206227E525BC
:1000C0006002E473E525F4C3334009758A00D26306
:1000D000F57C01D6F58A758B00758D00D262D0E073
:1000E000D0D0D2AF32C3E526334009758A00D2633F
:1000F000F57C01F6F58AC262E526F4603B306803C0
:10010000207213758B00758D00D0E0D0D0D293D2C1
:1001100097D295D2AF32D293D297D295206E0C203F
:1001200066097410D5E0FDE57E4290758B00758DF3
:1001300000D0E0D0D0D2AF32758A00D263757C0097
:10014000C28DD262212B01C4306805206602C293A1
:1001500001C4306805206602C29501C430680520DC
:100160006602C29701C4C29230680A2066077416FC
:10017000D5E0FDC29301C4C29430680A20660774BA
:1001800016D5E0FDC29501C4C29630680A20660704
:100190007416D5E0FDC29701C4C2AFC2AD53E6EFFD
:1001A000C0D0C0E0D2D3D2AFE57D6009E57A60056A
:1001B000757A00413E757A01C2CEE52A6007207447
:1001C00049152A410A7800790020742EE580307E96
:1001D00001F430E50278FF53DACF207E0343DA20C2
:1001E000307E0343DA10C2D8C271E580307E01F45C
:1001F00030E50279FFC3E89970CB306103752A407E
:10020000207403752A40885FD27020740DE52B603E
:1002100004152B411A43DA01C2D8207002412DA8DF
:100220005F206102C270207402412B88227882B65E
:100230000403852224C3E52594404002D26420CFE4
:100240000AD0E0D0D043E610D2AD32C2CF053AE5B5
:100250007D6009E57B6005757B00612B757B01780E
:1002600002E52A6005307402152AC3E55F94014057
:10027000057562004187756300756C00E5622401B5
:10028000F56250037562FF7982B7020D306D1DC3B0
:10029000E52294324016854D227982B7030E306DE7
:1002A0000BC3E52294324004798E8722C3E523955F
:1002B0002260084004152341BB0523D8CA056CE51C
:1002C0006C7002156CD56D63756D017805C3E56CB6
:1002D000956E4057C3E56C956F50087801756D03B6
:1002E0000202EFC3E56C957050057801756D01C38E
:1002F000E5659524401E7982B704026120206D14C3
:10030000852465E56C046003856E6C756D0175234D
:100310003C02032BE5652850057565FF6120F565F6
:10032000E5650470067563FF756CFFD0E0D0D043BF
:10033000E610D2AD32C2AFC0D053E67FC260759135
:1003400000855694855795759104D0D0D2AF32C2AE
:10035000AF53E6EFC2ADC0D0C0E0C0F0D2D3D2AF51
:10036000A8FBA9FCE57D6007C3E913F9E813F8C20F
:10037000D830710261C153DACF207E0343DA1030E6
:100380007E0343DA20D271E580307E01F420E5025D
:10039000619888278928A1A053DACF207E0343DA09
:1003A00020307E0343DA10C2D8C271307402A18CAF
:1003B0007800E580307E01F430E502A18C885FA1F1
:1003C0007453DACF207E0343DA20307E0343DA1001
:1003D000C271206102819A53DACF207E0343DA1082
:1003E000307E0343DA20C2D8D271885A895BC3E8D1
:1003F0009558F8E99559F97B007E087A00C3E8948E
:100400008CE994005005755E00818C882178A2E605
:10041000A8216055C3E894C8E994005008E4D2E4E8
:10042000FB7A0A8167C3E89468E994015008E4D232
:10043000E3FB7A0F8167C3E894D0E994025008E4A3
:10044000D2E2FB7A1E8167C3E894A0E994055008C4
:10045000E4D2E1FB7A3C8167C3E89498E9940850C0
:1004600008E4D2E0FB7A787E00C3E8955CFCE9956D
:0F0470005DFD30E70AECF42401FCEDF43400FDEF
:10047F00755E00C3EC9AED9E5003755E01885C8932
:10048F005D855A58855B597802A174C3E89527F8A2
:10049F00E99528F9307C02A158307B02A158307AB7
:1004AF0002A15120750281BDE9FDE8FC81DCE9C3A1
:1004BF0013F9E813F8307902A151E9C313F9E813DE
:1004CF00F8307802A151E9C313FDE813FC2061262F
:1004DF00C3EC941CED9402400281F3ED7018C3EC51
:1004EF0094C850120529C3E529940A5002A18C75AE
:1004FF005F00D270A18CE529600215297400207F5E
:10050F00037896E624FAFEE43400FFC3EC9EFCED7C
:10051F009FFD500678007900A158C3EC94FFED942D
:10052F0000400678FF7900A158EC8575F0A4C5F05E
:10053F00A2F733F87900400302057478FF790002BF
:10054F000574E9C313F9E813F8307C0EE9600278FB
:10055F00FFC3E81338F8E43400F9C3E894FFE994D3
:10056F0000400278FF885FD270206102A18C741F57
:10057F00F4552F4BF52FC274EB7002D274752A40CD
:10058F00307403752A0A306102A1A020740353DA74
:10059F00FE207403752B20D0F0D0E0D0D0D2AD4325
:1005AF00E6103279010205D079030205D0790A02EB
:1005BF0005D0791E0205D079640205D079C80205ED
:1005CF00D07817E4D5E0FDD8FAD9F6227A147B78E3
:1005DF000205F77A107B8C0205F77A0D7BB40205C2
:1005EF00F77A0B7BC80205F77902B27DE4C294D586
:1005FF00E0FDC295D5E0FDD295D5E0FDD294D5E0D2
:10060F00FDC293E576D5E0FDD2937496D5E0FDD982
:10061F00D9EAF8D5E0FDD8FBDBCEC29422C37C002B
:10062F007D0075F00005F0EA33FAEB33FB50F6EB83
:10063F0013FBEA13FAC3E9FFE8FEE89AF8E99BF91E
:10064F005004EFF9EEF8B3EC33FCED33FDD5F0DFEA
:10065F00EDF9ECF822E889F08A20D2D4F8A9F07BE2
:10066F000030F70B7BFFF42401F8E9F43400F9E8CC
:10067F008520F0A4ADF0F8E98520F0A4AFF0FEEDF1
:10068F002EF974003FFA7C04C3EA13FAE913F9E870
:10069F0013F8DCF48BF030F70AE8F42401F8E9F4EE
:1006AF003400F9E889F0C2D4F8A9F0227882B604B0
:1006BF000302075AC3E55F9419401EE52D540670D7
:1006CF0018206D3678057994E7146007780A14605E
:1006DF00027812C3E54198401F306D098567657533
:1006EF006CFF756D01852224E4F545F546F547F558
:1006FF0048F549C26D02075AD26D7994E714701309
:10070F00E523F43333F913F8E9540104F9E854FEFF
:10071F0002074EE714147014E523F4333333F9133F
:10072F00F8E9540304F9E854FC020756E523F433BF
:10073F00333333F913F8E954070404F9E854F8C3D1
:10074F009440F8E99400F98845894622C3E541139E
:10075F00F9E54013F8C3E54598F8E54699F9500CCB
:10076F00C3E89480E994FF4016020792C3E8947F90
:10077F00E994005003020792787F7900020792787C
:10078F008079FF884A894B22E54A2547F8E54B35A2
:10079F0048F9854B20E4300701F43549FA30E70971
:1007AF00C3EA94F040150207D0C3EA940F50030236
:1007BF0007D078FF79FF7A0F0207D0780079007A97
:1007CF00F0C3E5249564500AC374019524500B02BD
:1007DF0007EEE54B20E70E0207EEE54B30E7068804
:1007EF004789488A492278A4E6FAC3E54A33F8E5EF
:1007FF004B33F9120664E930E70BC3E89480E994B0
:10080F00FF40130129C3E8947FE9940050020129A6
:10081F00787F79000129788079FFE820E715C3E513
:10082F002398F84009C3E894014003020850780167
:10083F00020850E8F424012523F8400302085078F9
:10084F00FF884C2278A5E6FAA848A949120664E960
:10085F0030E70CC3E89401E994FF4016020885C302
:0F086F00E894FFE99400500302088578FF7900B0
:10087E00020885780179FFE920E715C3E54C98F861
:10088E004009C3E8940140030208AC78010208ACA9
:10089E00E8F42401254CF840030208AC78FF8824C4
:1008AE002278FFC26420693D206A12D264C3E541FA
:1008BE00940A4009C3E52594405002C26479A1E729
:1008CE006023E541601F74FF8541F0848539F03067
:1008DE006A0375F005A4F8C5F0600278FFC3E895C9
:1008EE00675002A867886622C3E54094C8E5419424
:1008FE0000E5665003142107046002F56622788332
:10090E00E6F520120FC475E8901205B275E890E571
:10091E00E820ECFBA8BDA9BE12105E7571007572C1
:10092E0000C3740013FD7400606613FC74002CFC8D
:10093E0074003DFDECFAEDFBC3E89AE99B4014E52B
:10094E00712400F571E5723400F572EA2CFAEB3D74
:10095E00FB80E5AE71AF72C3E57213F9E57113F862
:10096E00C3E913F9E813F87A03C3E913F9E813F8A6
:10097E00DAF7AA201A700975710075720002099EC5
:10098E001AEA6008EE28FEEF39FFDAF88E718F72E0
:10099E002275E890227883E6FFE5E820ECF7A8BD03
:1009AE00A9BE0573C3E57394084052757300E9FA46
:1009BE0079A0E76044EA7007E574601B0209D9C3A9
:1009CE00E895746010E5745006600C140209E50495
:1009DE0060F90209E5E574F574C39472401B756401
:1009EE00C0C394044013756480C39404400B7564B3
:1009FE0040C39404400375640075BB0822EFC39492
:100A0E0001601F7400601BC3E894FFE99403501249
:100A1E00C3E89571E995725009E564600C1564029E
:100A2E000A37E564F460020564A864C3E5249850AF
:100A3E0002A824C3E89565400AA865E565F460033D
:100A4E0085656488258826E573B4070375BB102277
:100A5E00743279A687F0A4C5F0A2F733F8C3E895EF
:100A6E00644002A864882288248825882688672204
:100A7E007540007541F022C2AF75C820A8CCA9CD33
:100A8E00AA3A30CF010A75C824D2AFC3EA13FAE9E5
:100A9E0013F9E813F8AB3BAC3C883B893CC3E89BAD
:100AAE00F8E99C20690A547FF930670261A8610554
:100ABE00AD3D8A3DF9EA9D547FFA600478FF79FFD7
:100ACE00AE3EAF3F8B3E8C3FC3EC9FFCC3E99CF523
:100ADE0042A83BA93CC3E89EF8E99FF9C3E5411340
:100AEE00FBE54013FAE82AF540E93BF5415006755F
:100AFE0040FF7541FF614FAA40AB41AC40AD417E16
:100B0E00047F02C3EB940440021E1FC3EB94084003
:100B1E00021E1FC3ED13FDEC13FCDEF7C3EA9CFAB5
:100B2E00EB9DFBEF6009C3E913F9E813F8DFF7EA71
:100B3E0028FAEB39FB8A408B4150067BFF8B408BAA
:100B4E0041C3EB94025002D2673069047F03617A8D
:100B5E007892E6FFC3E537948240110FC3E53794D0
:100B6E00A040010FC3EF940640027F057E03E541CE
:100B7E00C4540FF9E541C454F0F8E540C4540F28AD
:100B8E00F8C3E89EFAE99400FB4009C3EA9402EB2D
:100B9E00940050047A02E4FB61F4AA40AB41EBC42A
:100BAE00FEEAC4540F4EFCC3EA9CFAEB9400FBC35E
:100BBE00E813C313F8EA28FAEB3400FB8A408B41A2
:100BCE00C3EB94024002C2677803EBC4FE7B00EADB
:100BDE00C4540F4EFAC3EA98FA4005C39402500269
:100BEE007A027892E6FF30600261F48552568553A0
:100BFE0057D26043E680C3E49AF8E49BF9C3E83326
:100C0E00F8E933F93067028195E8FAE9FBD3E91385
:100C1E00FDE813FC88528953C3EF94036038EF202C
:100C2E00E00DE82CF8E93DF9ECFAEDFB020C50E88A
:100C3E0028F8E939F9C3E82402F8E93400F97AFE14
:100C4E007BFFC3EF9403400E8A548B55884E894F19
:100C5E008C508D5181C9885489558A4E8B4F8C503A
:0E0C6E008D51306920C3E53394034019E542EF
:100C7C00A2E713F8E555F4240138400B20E708757A
:100C8C0054FFF42401F55581C9E8FAD3E813FC8824
:100C9C0052C3EF94036020EF20E007E82CF8ECFA45
:100CAC0081B5E8282402F87AFEC3EF940340088A41
:100CBC0054884E8C5081C988548A4E8C50E56BC335
:100CCC00335002646BF56B30600281D3753404D2FF
:100CDC006043E680E52D5406601FA840A941C2AFD1
:100CEC0053E67F759100C3E498F594E499F59575F6
:100CFC009104D26043E680D2AF22D2657544007570
:100D0C002000306B03752040020D25D26575440020
:100D1C00752040306B03752000D2AF78012067221C
:100D2C00E52D54066002C265C3E541940540137875
:100D3C000294054008780394054002780630690255
:100D4C00780A206019E544601530690AC3E53394CC
:100D5C00034003D53406D2AFD26CC10791DBD2AFBE
:100D6C000000C2AF20672AE541C3FB940F40027B11
:100D7C000FEB240530730123306A027428206201C2
:100D8C0023F93069027982E58D13E58B13C3994001
:100D9C00B10544E59B5440B52002A1F130690A0825
:100DAC00C3E8940A400108A14E206502A125C26542
:100DBC0053E67F7591003067107594007595FC753E
:100DCC009104D26043E680A125AE40AF41C3EE331F
:100DDC00FEEF33FF50047EFF7FFFC3E49EF594E4E7
:100DEC009FF595A1CBC3E53394025002A125306544
:100DFC0002A125D802C105A14EC26C53E67F7591A4
:100E0C0000855494855595759104854E56854F579C
:100E1C00D26043E680D2AFE52D54066008206A020A
:100E2C000533020E41306C0D206B0A2065071581CD
:100E3C0015810216A3227800306405306502780112
:100E4C00E53775F007A4F9E5F028F5F0E9A2F01301
:100E5C00A2F113A2F213F537C394785003753778C7
:100E6C00C3E53795384008D266D293D297D29530E5
:100E7C006002C17B855056855157D26043E6802273
:100E8C00207D11C2AF754302C294D292D2AF759F2E
:100E9C004002105BC2AF754302C294D296D2AF75BA
:100EAC009F4002105B307243207D20C2AF7543031C
:100EBC00900177757E10D297C296306204C295C1AC
:100ECC00CFD294D2AF759F4102105BC2AF75430372
:100EDC00900177757E10D293C292306204C295C194
:100EEC00EFD294D2AF759F4302105B207D17C2AF37
:100EFC00754303900152D297306202C295D2AF75FE
:100F0C009F4102105BC2AF754303900152D29330E4
:100F1C006202C295D2AF759F4302105B207D11C255
:100F2C00AF754304C292D296D2AF759F4302105B49
:100F3C00C2AF754304C296D292D2AF759F410210D4
:100F4C005B307243207D20C2AF75430590016675FE
:100F5C007E04D295C294306204C293E16BD292D2D9
:100F6C00AF759F4002105BC2AF7543059001887549
:100F7C007E40D295C294306204C297E18BD296D255
:100F8C00AF759F4002105B207D17C2AF7543059073
:100F9C000148D295306202C293D2AF759F400210C5
:100FAC005BC2AF75430590015CD2953062EBC29782
:100FBC00D2AF759F4002105B207D11C2AF75430606
:100FCC00C296D294D2AF759F4102105BC2AF7543EB
:100FDC0006C292D294D2AF759F4302105B3072421C
:100FEC00207D20C2AF754301900188757E40D2935D
:100FFC00C292306204C2970107D296D2AF759F435A
:10100C0002105BC2AF754301900166757E04D297E6
:10101C00C296306204C2930127D292D2AF759F411F
:10102C00015B207D16C2AF75430190015CD29330F9
:10103C006202C297D2AF759F43015BC2AF75430189
:10104C00900148D297306202C293D2AF759F41C2D1
:10105C006622900146757E00D293D297D295C292A9
:0F106C00C296C294C2622278807607087607087F
:10107B0076010876040876FF0876FF08760B08766B
:10108B0002087601087601788C76010876000876DE
:10109B00B40876FF0876FF0876FF0876030876FF1C
:1010AB000876010876FF0876250876D0087678084A
:1010BB0076C80876040876FF08760108760008766D
:1010CB007A0876070876010876010876000876FF1D
:1010DB00227887E6FFC272BF0302D2727888C27D84
:1010EB00E630E102D27DC27E7889E630E102D27E23
:1010FB00C3EF94026008758E01D27302110E758EC8
:10110B0000C273227880E6149000809378A4F6785E
:10111B0081E6149000809378A5F67886E61490000B
:10112B008D9378A6F6789FE6F8700108C3E89411C2
:10113B0040027811E82828F56E256E256E28F56F8C
:10114B00256E2828F570789CE67538FF75390CB438
:10115B0002067538A075390AB403067538827539DD
:10116B000578A3E61490009A93F569115E22227814
:10117B0096E6FA7897E6FB7888E6B40305C3EB941A
:10118B000EFB307F047A007BFFC3EB9AFCC3948287
:10119B0050027C827575000575EC8575F0A4C3E56E
:1011AB00F0947D40F222D27F317A1205C17A007B16
:1011BB00007C101205B7E55F2AFA74003BFBDCF3E9
:1011CB007C04C3EB13FBEA13FADCF7FEC27F317A24
:1011DB0022E5EF20E6037520000520903FFFE52078
:1011EB00146006901FFF1460009304600375EF12E8
:1011FB0053D9BF7581C043FF801205B275EF02430F
:10120B00B203E5B3240420E70DF521E5E320E00666
:10121B008521B343E301115E7580FF75A40075F161
:10122B003075D4DF7590AB75A5FC75F2FC75D501E7
:10123B0075A60175E241E4F8F6D8FD756B011173E3
:10124B001216F278988676753001C2AF1205CB1262
:10125B0005DB1205C11205E21205C11205E91205E3
:10126B00C11218141205CB1205CB1205C6C2AF78EA
:10127B00FA79FA308507D9FBD8F7021C0011DC315B
:10128B000F3179317A78988676115E75B68075A9AB
:10129B0000757D0075885075891275C82475910489
:1012AB0075D84075A82275B80275E690759B807548
:1012BB009D0075D10E75BC5875BB0875BA1175E8D4
:1012CB00801205B2D2AF12090C53DACF207E034342
:1012DB00DA20307E0343DA1043DA01C2D8C271122E
:1012EB0005CBD2617B037A0CE55E70077A0CDB03CE
:1012FB000212781205C1207003021278C270E55FEA
:10130B00C3940240E1E52F541F856160F561B56020
:10131B00D5DAD5C26153DACF207E0343DA20307E93
:10132B000343DA10C2D8C27178A2E67008D274E512
:10133B002F54E0F52FC2757529001205C6307409BC
:10134B00C3E529940A4002D2751205B778023074AE
:10135B00027800C3E55F9840F0C2AF1205DB1205BF
:10136B00DB1205DBD2AF1205CB754D001205B7783A
:10137B008CE6C39401500302144DE530C394015025
:10138B000302144D207435C3E55F94FF5003021420
:10139B004DC2AF1205F0D2AF1205C6C3E55F940183
:1013AB0050EFC2AF1205DB1205BC1205DBD2AF1238
:1013BB0005C6C3E55F94FF40E90218997F05D27F0C
:1013CB00317A1205C6C2AFC27F317AAE5FC3E55F19
:1013DB00947FD2AF40761205B2C2AF1205F0D2AFF6
:1013EB00DFDC31B1C3EE94057897F61205CB1217FB
:1013FB003312181C7F0AD27F317A1205C6C2AFC2D4
:10140B007F317AAE5FC3E55F947FD2AF50E61205B2
:10141B00B2C2AF1205DB1205BC1205DBD2AFDFD6B1
:10142B0031B1EE24057896F61205CB12173312184C
:10143B004B1205C6317AC3E55F94FF5002618F02F0
:10144B001899C3E55F954D4003855F4D1205C6782E
:10145B00017988E7B403027805C3E55F9840026120
:0E146B0077C2AF1205F01205F01205F0D2AFF5
:101479001205CB753000E4F531F5320531E531F46B
:1014890070390532789AE678191460127832146046
:101499000D787D14600878FA146003753200C3E58D
:1014A9003298401715327531B478998676C2AF12E1
:1014B90005F0D2AF789886761205C61205BCE52AE2
:1014C9007005307402417878012074027806C3E50A
:1014D9005F9840A71205C6E52A7003021278C2AFC9
:1014E900115EE4F522F523F524F525F526F56AD2F2
:1014F900AF7885E6C333F568E4F545F546F547F574
:1015090048F549F573F52CF52DF53775730875BB55
:10151900101205B212099FE5E820ECFBA8BDA9BE8F
:10152900E97001F888741209A375730875BB1078FE
:1015390087E6FE760211DC7887EEF6C2AF7564FFA6
:10154900120A5E852264852265852266D2AF7522DC
:101559000175240175250175260185636C756D0179
:1015690075B69075A903757D017888E6B40307C23D
:101579007D307602D27DD268D269753300120FC4EC
:10158900120FE9120A7E120A85120A7E120A8512C0
:101599000A7E0215AAC2AF11DCD2AF75730075BB02
:1015A90008120D171206BB120E42120E8C120A8572
:1015B900120D06306D0312075B2067031208AF3066
:1015C90067031208F6120E42120EB1120A85120DA5
:1015D90017306D03120797120E42120F28120A854F
:1015E900120D06306D031207F5120E42120F4D123D
:1015F9000A85120D17306D03120853120E42120F8D
:10160900C4120A8512099F120D06120E42120FE921
:101619001209A3120A8530692F206B2C856764850E
:10162900676585636C756D0179187A0CC3E5339923
:101639004009C269D26A8A35021651C3E55F94012D
:1016490040030215AA0216AB306A1B206B18E53558
:10165900147004C26AA19EF535C3E55F9401400385
:101669000215AA0216AB753600C3E562940140095A
:1016790085676585636C756D01C3E56278FA985075
:1016890021307404E52A601A78F0306B05856764A7
:101699007820C3E541985002A1AA0536E55F6002AA
:1016A900C1AE753600C2AF115E7887E6FE760211CB
:1016B900DC7887EEF6E4F522F523F524F525F52601
:1016C900F568C26875B68075A900757D00D2AF123C
:1016D90005B2115E307406E52A70024178788DE60C
:1016E900C3940140026154817F901A0D782012172A
:1016F90075E520B4A50CA3121775E520B45A0302A9
:1017090017131173121733021732901A0378807B5B
:101719000A121775A308DBF9901A0F788C7B181237
:101729001775A308DBF9901A2722C2AF1217B41252
:10173900178E901A00740E12177AA3740412177A6E
:10174900A3741412177A901A0378807B0A121779F6
:10175900A308DBF9901A0F788C7B18121779A30864
:10176900DBF91217C71217A5901A2722E493F6225C
:10177900E6438F01538FFD75EF0275B7A575B7F174
:10178900F0538FFE22438F02438F0175EF0275B725
:10179900A575B7F1901A0DF0538FFC22901A0D74AC
:1017A900A5F17A901A0E745AF17A227A3079D078A2
:1017B90020901A40F175E520F709A3DAF7227A306B
:1017C90079D0901A40E7F17A09A3DAF922AB77A820
:1017D90078BB01027980BB02027981BB030279825D
:1017E900BB04027994BB05027983BB06027986BBE7
:1017F90007027992BB08027987BB0902799CBB0A67
:10180900027988BB0B027989E8F7227C051205CB9E
:10181900DCFB22C2AF1205DB1205E21205E9120553
:10182900F01205BC1205DB1205E21205E91205F0FA
:101839001205BC1205DB1205E21205E91205F0D208
:10184900AF22C2AF1205F01205E91205E21205DB5B
:101859001205BC1205F01205E91205E21205DB12A8
:0E18690005BC1205F01205E91205E21205DBBE
:10187700D2AF22AE77AF78C2AF1205DB1205DB120B
:1018870005DB1205BCDEF21205F01205BCDFF8D24B
:10189700AF22111C11141114757701757801757930
:1018A70000117A7C05AD5F1205CBC3ED955F70F52E
:1018B700C3E55F9401400AC3E55F94FF4034021813
:1018C700D71217D6121733111CC2AF75EF121114A6
:1018D700DCD30579C3E5799403500280C41114055C
:1018E70078E5771490009F93F808C3E5789850023D
:1018F70080AC111411140577C3E577940C5002805E
:0E1907009A121073121733C2AF75EF1211143B
:0319FD000211DCF8
:101A00000E041407070104FFFF0B020101A55A0190
:101A100000B4FFFFFF03FF01FF25D078C804FF01DA
:081A200000FF07010100FFFFB8
:101A40002358526F746F72313041232020202020A0
:101A500023424C48454C492346333930232020202B
:101A60002020202020202020202020202020202076
:101C0000C2AFC2D353D9BF7581C043B20343FF8073
:101C1000752438752503B1C975EF0275E24043F1AB
:101C20002053A4DF75D400D2857DFA780379E67C51
:101C300010752200752300901DD67B0675249875BB
:101C400025013085028142208508D8FBD9F9DCF7CF
:101C500081B4308508D8FBD9F9DCF781B4B189E4C7
:101C600093A3C39A6004DDC381B4DBDBB17B600264
:101C7000812B7B08E493FAA3B15CDBF87A30B15C8A
:101C8000752200752300B17BEAFCEBFDC3ED94FEE9
:101C9000400EB17B8A278B28ED30E0048A828B834B
:101CA000B17B7AC270D8C3ED94FE601350CEBD00F4
:101CB00025EC60097520007521FF0200008100A855
:101CC00027A9280809D804D90281D3B17FEA89AAB3
:101CD000F281C50D81A0C3ED94035049EDA2E092BD
:101CE000007AC5C3E5829400E583941C50902000DF
:101CF00010438F02438F0175B7A575B7F1F030001F
:101D00001FA827A9280809438F01538FFDD804D99C
:101D100002A12089AAE275B7A575B7F1F0A3A10DBC
:101D2000538FFC817C7AC1BD030CE493A3FAB140CC
:101D3000DCF8B138817C817EAA22AB23B15CEBFA5E
:101D4000EA6222752608C3E52313F523E52213F57D
:101D50002250066323A0632201D526EAB1C9B1C986
:101D600075260AEAF4200102D285300102C285B14B
:101D7000C9C3134002C201D526EB22B17FEAFB2082
:101D80008502A17F308502A184752608AE24AF2587
:101D9000C3EF13FFEE13FEB1CDB1C9C3EA13308513
:101DA000024480FA30E703632201C3E52313F523DD
:101DB000E52213F52250066323A0632201D526D91C
:101DC000E52265236523F52222AE24AF250E0FDE22
:101DD000FEDFFCD20122424C48656C693437316326
:041DE000F390060175
:00000001FF
